:1000000000620000000B0000AC0A000000000000CD
:1000100000000000000000000000000000000000E0
:1000200078FFE4B8200118F6D8F99000007F007E30
:1000300007E4F0A3DFFCDEFA75817A022390121A3E
:10004000961220629002117401F022022C4E74AAC2
:100050007583F5758255A574557583FA7582AAA5C1
:1000600074A57583F5758255A52200021E5AEE30DF
:10007000E707C3E49FFFE49EFE2274BB2F122B9878
:10008000E4F02202191312109BE4F0A37402F02290
:1000900012109B7480F0A3E4F02200022C4BE709BD
:1000A000F608DFFA8046E709F208DFFA803E888228
:1000B0008C83E709F0A3DFFA8032E309F608DFFA60
:1000C0008078E309F208DFFA807088828C83E30984
:1000D000F0A3DFFA806489828A83E0A3F608DFFA5E
:1000E000805889828A83E0A3F208DFFA804C80D2AC
:1000F00080FA80C680D4806980F28033801080A628
:1001000080EA809A80A880DA80E280CA803389827F
:100110008A83ECFAE493A3C8C582C8CCC583CCF02B
:10012000A3C8C582C8CCC583CCDFE9DEE7800D89D2
:10013000828A83E493A3F608DFF9ECFAA9F0EDFBD9
:100140002289828A83ECFAE0A3C8C582C8CCC58321
:10015000CCF0A3C8C582C8CCC583CCDFEADEE8807A
:10016000DB89828A83E493A3F208DFF980CC88F0EC
:10017000EF60010E4E60C388F0ED2402B40400501D
:10018000B9F582EB2402B4040050AF232345822347
:100190009008CE73EF8DF0A4A8F0CF8CF0A428CEF9
:1001A0008DF0A42EFE22C2D5EC30E709B2D5E4C30F
:1001B0009DFDE49CFCEE30E715B2D5E4C39FFFE45F
:1001C0009EFE120BF2C3E49DFDE49CFC8003120B27
:1001D000F230D507C3E49FFFE49EFE22C5F0F8A3EA
:1001E000E028F0C5F0F8E582158270021583E0384A
:1001F000F022BB010A89828A83E0F5F0A3E0225055
:100200000687F009E71922BBFE07E3F5F009E319B9
:100210002289828A83E493F5F074019322BB01075B
:1002200089828A830209BC500B09C5F027F7C5F003
:100230001937F722BBFE0D09F8E325F0F3C5F019D5
:10024000E338F322F889828A8374019325F0C5F09C
:10025000F8E4933822BB010A89828A83F0E5F0A38F
:10026000F0225006F709A7F01922BBFE06F3E5F0CD
:1002700009F3192275F008758200EF2FFFEE33FEA7
:10028000CD33CDCC33CCC58233C5829BED9AEC996E
:10029000E58298400CF582EE9BFEED9AFDEC99FC10
:1002A0000FD5F0D6E4CEFBE4CDFAE4CCF9A8822257
:1002B000B800C1B90059BA002DEC8BF084CFCECD77
:1002C000FCE5F0CBF97818EF2FFFEE33FEED33FDB0
:1002D000EC33FCEB33FB10D703994004EB99FB0F95
:1002E000D8E5E4F9FA227818EF2FFFEE33FEED336C
:1002F000FDEC33FCC933C910D7059BE99A4007ECE4
:100300009BFCE99AF90FD8E0E4C9FAE4CCFB22752A
:10031000F010EF2FFFEE33FEED33FDCC33CCC833BE
:10032000C810D7079BEC9AE899400AED9BFDEC9A20
:10033000FCE899F80FD5F0DAE4CDFBE4CCFAE4C898
:10034000F922EB9FF5F0EA9E42F0E99D42F0EC6461
:1003500080C864809845F022EB9FF5F0EA9E42F059
:10036000E99D42F0E89C45F022E8600FECC313FCE5
:10037000ED13FDEE13FEEF13FFD8F122ECF0A3ED29
:10038000F0A3EEF0A3EFF022A8828583F0D083D013
:1003900082120B7F120B7F120B7F120B7FE473E430
:1003A00093A3C583C5F0C583C8C582C8F0A3C58320
:1003B000C5F0C583C8C582C822EC8EF0A4CCC5F0B8
:1003C000CCCDF8EFA4CEC5F02DFDE43CFCE8A42E86
:1003D000C8C5F03DFDE43CFCEFA4FFE5F028FEE4D9
:1003E0003DFDE43CFC22EF4E6012EF60010EEDBBE0
:1003F000010B89828A83F0A3DFFCDEFA2289F050A8
:1004000007F709DFFCA9F022BBFEFCF309DFFCA91A
:10041000F022BC000BBE0029EF8DF084FFADF0226E
:10042000E4CCF875F008EF2FFFEE33FEEC33FCEE72
:100430009DEC984005FCEE9DFE0FD5F0E9E4CEFD65
:1004400022EDF8F5F0EE8420D21CFEADF075F00838
:10045000EF2FFFED33FD4007985006D5F0F222C391
:1004600098FD0FD5F0EA22208A03020FCF900214E4
:10047000E07002A3E06003020FCF900171E0700210
:10048000A3E06003020FCF12114E6003020FCF9062
:100490000132E0703090011D120FE4FFAEF09001C8
:1004A0000B120FE4D39FE5F09E4003020FCF121012
:1004B0004AE490017DF0A3F01211C19002181211CC
:1004C000D8F5758003757500757616E4F5B2F5BA42
:1004D000900181E0F55DA3E0F55EC209758D2043D2
:1004E0008D20758D8043AA08D2AF758B02758EAFB3
:1004F00020062412114E701F200C1CE5DB20E21791
:10050000758AC4200C0DE5DB20E208758703000026
:10051000008006D2098002D209758B11758A50536A
:10052000AAF7D3900213E09490900212E094014055
:100530000EA3E02470F0900212E034FEF08007E495
:10054000900212F0A3F0D390021FE0949090021E4C
:10055000E09401400EA3E02470F090021EE034FE0F
:10056000F08007E490021EF0A3F0122A3E9000559E
:10057000E075F006A4902EC3F0A3E4F0A3F01210EF
:100580002153997F1208661210C2902EC0E030E20B
:10059000F9902EC0E4F0902E02E0F577A3E0F57814
:1005A0004389021210274380021210BF902EC0E030
:1005B00030E2F91211ECF522A3E0F523E5782527C6
:1005C000FFE5773526FEC3EF9523F525EE9522F559
:1005D00024121196E5259FE5249E40048E248F2544
:1005E000902EC4E4F043998090016FE524F0A3E5D8
:1005F00025F0C3E55E9525FFE55D9524FE12084EC6
:100600008E5F8F601211FF4003020FA8AE24AF254A
:100610007C007D14120B99121209AF74AE73AD7287
:10062000AC719002C4121007FBD3120B389002C4B5
:1006300040171211009574FFEE9573FEED9572FD53
:10064000EC9571FC1212098007120B680000000083
:10065000E47F607EEAFDFC9002C4121007FBD31217
:100660000B38400A9002C4120B680000EA60120FB7
:10067000E1FFAEF07C007D09120B999002C41210CC
:10068000072FFFEA3EFEE93DFDE83CFC1211721225
:100690001209900132E07033AE5DAF5EFC7D09124D
:1006A000112DE4FCFDEB2525FFEA352412106C1218
:1006B00011728E5D8F5E9002C4120FF2121036120C
:1006C00010F2120FFC121036020FA81210F2120FC5
:1006D000FC12103690010E120FE4FFAEF09002C42F
:1006E000121004FBD3120B385003020FB8120FD0B4
:1006F000121147FEC3EF957AEE95795003020FB8B9
:1007000090010B120FE4FFAEF07C007D02120B99FA
:10071000C8ECC8EDC0E0EEC0E0EFC0E0120FD012B0
:100720001147FEE4FCFDD0E0FBD0E0FAD0E0F9EBAD
:100730002FFFEA3E12106C7B0312117490010B1212
:100740000FFC1210B890010B120FE4D39430E5F0B7
:1007500094754008747575F030120A35900184E084
:100760006066121155406190010B120FE41211479F
:10077000FE12084E9002C8EEF0A3EFF090010B12AB
:100780000FE4FFC312103E50199002C9E094149078
:1007900002C8E09400400B120FF9F9E475F005125D
:1007A00009FD900185E0602090010B120FE412100A
:1007B0003C4015D39002C9E094289002C8E0940010
:1007C0004006120FF91211F620090D1211FF500800
:1007D00012114E7003020CBC900183E0041211153B
:1007E0001210129001337401F090021612117B2244
:1007F00090010EE0FBA3E0FAA3E0F91209D2FFAEEC
:10080000F0900108E0FBA3E0FAA3E0F90209D2901E
:100810000134A3A3E0F9A3E0FF90010EE0FBA3E005
:10082000FAA3E022E4FCFDE0F8A3E0F9A3E0FAA3D8
:10083000E0227A0079667E007F0B7D007B00020B50
:10084000C643AB025389FD5395FD5396FD22A3F099
:10085000A37401F0A322C98FF0020A35D3FF9001DF
:1008600089E09F900188E095F0227F087A01793431
:100870007E007D007B01020BC6E50A25E02428F8F6
:10088000E6FE08E622F9EB2FFFEA35F0FEED39FD32
:10089000EC38FC229002147402F0A37458F022A3E6
:1008A000E0FEA3E0FBCAEECAE4F9F822902E427DF6
:1008B00014E0FEA3E0FF7C00020974902EC07402D5
:1008C000F0902EC27412F0902EC77401F0902EC4D6
:1008D00022F9E4F5F0020A35F9EE8FF0020A35123A
:1008E0000870902EC07419F022E50D25E02475F5EE
:1008F00082E43401F583E0FEA3E0FF229002C6E02B
:10090000FEA3E0FF2290018AE0FCA3E0FDC3EF9D7F
:10091000FF229002C4A3A3E0F9A3E0FF9001082204
:10092000E0FCA3E0FDA3E0FEA3E022900186F0A39B
:10093000F0A3F0A322F07E007F057D007B007A000B
:100940007961020BC6FFE5F0F0A3EFF022120B99DC
:10095000C8ECC8C9EDC9CAEECACBEFCB22E4F50E8C
:10096000F50DF50CF50B22C39FFFE5F09E229000DC
:100970001BE0642022900188E0FEA3E0FFD39400F6
:10098000EE940022902EC07402F0902EC4E4F0A3E6
:10099000F0227B0AE4FAF9F8020A90E4F0A374C8A2
:1009A000F022AB0EAA0DA90CA80BD3020B387402CF
:1009B000F0A374BCF022E5272488FFE5263413FE5B
:1009C000D3227403F0A374E8F02290016FE56CF079
:1009D000A3E56DF02225E02428F8A60F08A6102232
:1009E000E490021AF0A3F022F9746175F0A8020AEB
:1009F0003590003A7410F022F0A3F0900220F0A39A
:100A0000F022FEEF2401FFE43EC31322902EC0E447
:100A1000F0902E1EE022F974FF75F0FB0209FDC371
:100A2000E5609576E55F9575229002C4020B5C90B7
:100A3000018C121007FBE9C0E0EAC0E0EBC0E090D7
:100A40000123120FE4FFE4FCFDD0E0FBD0E0FAD07C
:100A5000E012106590018C120B5C900191E004F0A3
:100A60007006900190E004F0900192E07002A3E023
:100A700060030213DA90018C121100FFEEC0E0EF68
:100A8000C0E012107FD0E0FFD0E0FE120A9090018B
:100A90008C120B5C90018CA3A3E0FFA3E090018A71
:100AA000CFF0A3EFF0A3120B6800000000E4900168
:100AB0009012110E74C8F0900212E07002A3E06070
:100AC000030213DA900132E0700302136990018689
:100AD000E0FEA3E0FF4E702290018AE0FDA3E090CB
:100AE0000186CDF0A3EDF090010B120FE4FD900113
:100AF00088E5F0F0A3EDF00213521210E5EE9CFE33
:100B000012084E900198120FFC1210B8900184E068
:100B10007026900198120FE4C3940CE5F0940050F5
:100B20000F90010B120FE4FF900188121126802014
:100B30009001847401F08018900198120FE4C3941E
:100B400002E5F094005009E412110BF0900184F0DA
:100B500090018AE0FEA3E0FFD3900187E09F90011F
:100B600086E09E4007E4900185F080069001857440
:100B700001F0E4900194F0A3F090019EF090019BAD
:100B8000120FFC1210B10213DA900194E0FEA3E000
:100B9000FF4E701590018AE0FDA3E0900194CDF026
:100BA000A3EDF0A31211A280511210E5EE9CFE12EB
:100BB000084E90019B120FFC1210B8900196E07045
:100BC00002A3E0703590019B120FE4D39419E5F075
:100BD0009400400C9001967413F0A37488F0800B7D
:100BE000E490019EF09001961211A290018AE0FF1C
:100BF000A3E0900194CFF0A3EFF0900132E07008F1
:100C000012110BF0900184F022120FD0FDACF0D342
:100C10009FEC9E403490010E120FE4FFC3ED9FFF46
:100C2000EC95F0FED3EF9430EE9475400D9002C633
:100C30007475F0A37430F002146C120FDB121147BC
:100C40009002C6F0A3EFF08043120FE1FFAEF090E8
:100C5000010E120FE4FDACF0C39FFFEC9EFED3EF3C
:100C60009410EE9427400C9002C674D8F0A374F050
:100C7000F08012120FE1FFC3ED9FFEEC95F09002A1
:100C8000C6F0A3CEF0E49002C6F0A3F0900132E0EB
:100C900060501210DCD39400EE64809480401A906F
:100CA0000120120FE4FDD3EF9DEE95F0400B900272
:100CB00018E4F0A37464F0801BD3900219E0940050
:100CC000900218E09400400C90010B120FE4900287
:100CD000C6121125D20B90021E740FF0A374A0F05F
:100CE000800D90021C1211A27A007952121016D3B4
:100CF0009002C7E094009002C6E0648094805003A4
:100D0000021593E0F9A3E0FF90010B120FFC121003
:100D1000361210DCEE3395E0FDFCE47BB87A88F9FE
:100D2000F8C3120B22500A9002C67488F0A374B85C
:100D3000F0D390021BE0940090021AE09400500758
:100D400090001BE0B4201D1210DCC39496EE64806A
:100D500094805010EF9400EE6480948040257C00D5
:100D60007D0A801430001C1210DCC394A0EE648055
:100D7000948F500F7C007D321209869002C6EEF0EF
:100D8000A3EFF0900132E0600C90021CE07002A32F
:100D9000E0700280009002C6E0F9A3E0FF90011429
:100DA000120FFC121036900114120FE424A8FFE574
:100DB000F0801D90010B120FFC1210B19001141263
:100DC0000FFC1210B19002C7E024A8FF9002C6E009
:100DD0003461F9900111120FFC12103622121164C5
:100DE00053997FF50BF50CF50DF50EF50A12086613
:100DF0001210211210C2902EC0E030E2F9902EC0E5
:100E0000E4F0438902121027438002902E02E0FE94
:100E1000A3E0250CF50CEE350BF50B1210BF902E50
:100E2000C0E030E2F91211ECFEA3E0250EF50EEE63
:100E3000350DF50D050AE50AC3940640B0439980C7
:100E4000902EC5E4F0E527240CFFE52634FEFED302
:100E5000EF950CEE950B4015900171E07002A3E048
:100E6000701290017104F0A374F4F08007E4900113
:100E700071F0A3F0E50C2527FFE50B3526FEC3EF47
:100E8000950EF510EE950DF50F121196E5109FE5F4
:100E90000F9E40048E0F8F10900167E50FF0A3E5C1
:100EA00010F090016BE50DF0A3E50EF0A3E50BF05B
:100EB000A3E50CF0AF10AE0F1221EB90016FEEF036
:100EC000A3EFF090001BE0B4200312101290016F0A
:100ED000E0FEA3E0FFE4FCFDE5692FF569E5683E6F
:100EE000F568ED3567F567EC3566F566056BE56B1E
:100EF0007002056AC3E56F94E8E56E9403402AAE7C
:100F00006AAF6BCBEFCB121085AF69AE68AD67AC43
:100F100066120A908E6C8F6DE4F569F568F567F5D9
:100F200066F56AF56BF56EF56FD3E56D9400E56CCB
:100F300094004059900170E0956DFF90016FE0952D
:100F40006CFE9002CAF0A3EFF0D394F9EE648094A3
:100F50007F4015E094079002CAE0648094805008B6
:100F60001211AAE4F57080259002CAE0FEA3E0FF0A
:100F700012084ED3EF9414EE648094804003757091
:100F800003E570C3940350051211AA057090016F18
:100F9000E0F550A3E0F55178287C007D007B007AD5
:100FA00000792A7E007F2802094E900132E070030A
:100FB00002182712104A90021612118E900184E036
:100FC0007003021912121155500302191290010BED
:100FD000120FE4121147FE12084E9002C6EEF0A363
:100FE000EFF0D39496EE9400400CE4900184F090DE
:100FF0000186F0A3F022900185E0602090010B12A1
:101000000FE412103C4015D39002C7E094289002E0
:10101000C6E094004006120FF91211F690010B126F
:101020000FE4C312103D40030219129002C7E0946E
:10103000149002C6E094005003021912120FF9F93D
:10104000E475F0050209FD900134121007FBE9C0B8
:10105000E0EAC0E0EBC0E0120FE1FFE4FCFDD0E00D
:10106000FBD0E0FAD0E0121065900134120B5C90D6
:101070000139E004F07006900138E004F0900216A7
:10108000E07002A3E0600302191290013412110013
:10109000FFEEC0E0EFC0E012107FD0E0FFD0E0FE36
:1010A000120A90900134120B5C90010E120FE4248E
:1010B00032FFE435F0FE900134121004FBD3120B22
:1010C00038403F900212E07002A3E0703590019E1C
:1010D000E0702F200B2C90013BE004F07006900193
:1010E0003AE004F0D390013BE0940590013AE0949B
:1010F00000401E120FEF121036E490013AF0A3F0F8
:10110000800F120FEF121036E490013AF0A3F0C2F4
:101110000B900134120B6800000000E4900138F0DD
:10112000A3F090019EE0900216600412117B22123F
:10113000118E22C0E0C083C082C0D0D2AF90022501
:10114000E004F0D3900213E09400900212E09400C7
:10115000400CA3E024FFF0900212E034FFF0D390A3
:101160000215E09400900214E09400400CA3E024E7
:10117000FFF0900214E034FFF0D3900217E09400E7
:10118000900216E09400400CA3E024FFF0900216B9
:10119000E034FFF0D3900219E09400900218E0943C
:1011A00000400CA3E024FFF0900218E034FFF0D3DD
:1011B00090021BE0940090021AE09400400CA3E01F
:1011C00024FFF090021AE034FFF0D3900223E09461
:1011D00000900222E09400400CA3E024FFF0900273
:1011E00022E034FFF0D3900221E09400900220E04E
:1011F0009400400CA3E024FFF0900220E034FFF0C4
:10120000D390021DE0940090021CE09400400CA3D7
:10121000E024FFF090021CE034FFF0C3E56F94E897
:10122000E56E94035008056FE56F7002056EC3E527
:101230005B94E8E55A94035008055BE55B70020592
:101240005AD3900193E09400900192E09400400CF6
:10125000A3E024FFF0900192E034FFF0D3900197D7
:10126000E09400900196E09400400CA3E024FFF08D
:10127000900196E034FFF0D3900172E09401900168
:1012800071E09400400CA3E024FFF0900171E03481
:10129000FFF0D390021FE0940090021EE094004003
:1012A0000CA3E024FFF090021EE034FFF0D0D0D079
:1012B00082D083D0E0327E007FFF7D007B017A0008
:1012C0007904120BC69002D87400F0A37404F09055
:1012D00001C57401F0A37400F0A374B8F09001CBC1
:1012E0007401F0A37400F074AC1229F57400F0A33B
:1012F0007494F09001C87401F0A37400F0A374C654
:10130000F09001D17401F0A37400F074D21229F5A9
:101310007400F0A3741F1229F67401F0A37402F094
:10132000902DE0E493FF9002D8E0FCA3E0FDF5826D
:101330008C83A3EFF0900002E0FFED24041229CF8C
:10134000900001E0FFED24051229CF900003E0FF9B
:10135000ED24061229CF902DE2E493FFED24121222
:1013600029CF902DE3E493FFED24141229CF9001AF
:10137000DA7401F0A37400F0A3743CF0E4FF75F09C
:1013800002EFA42401F582E5F0342EF583E493FE08
:1013900074542FF582E43400F583EEF0EF25E02459
:1013A0002DF582E4342EF583E493FE1229FDEEF050
:1013B0001229FDE0FEEF25E0242CF582E4342EF521
:1013C00083E49324C0F582E4342EF583EEF00FEF2E
:1013D000B416AB902F56E0900058F0902F56E09046
:1013E000006EF0902F56E0900059F0902F56E0904C
:1013F000006FF09000FF7401F09000FEF090003A52
:101400007410F090001BF0900028F0A37420F0906E
:1014100002127413F0A37488F02212113DF515F531
:1014200016852811852912852813852914F50A1295
:101430001059FFD3E5149FE5139E40078E138F14B8
:10144000850A16C3E5129FE5119E50078E118F1273
:10145000850A15050AE50AB414D5E4F50FF510F56B
:101460000AE516650A602EE515650A6028E510454F
:101470000F7010E50A25E02428F8E6F50F08E6F5D8
:101480001080121210592510FFE50F3E1211E2F5DF
:101490000FEF13F510050AE50AB414C5900181E5B4
:1014A0000FF0A3E510F0E516C394115005E51612F0
:1014B00011B5E515C394115005E5151211B51211BA
:1014C0003DF50A121059FFC3E5109FFFE50F9EFE80
:1014D00012084ED3EF9419EE64809480400FE4FC20
:1014E000FDE50E2510F50EE50D350F800F12105994
:1014F000FFE4FCFDE50E2FF50EE50D3EF50DED3597
:101500000CF50CEC350BF50B050AE50AC3941440F9
:10151000B2AF74AE73AD72AC71121182401AE50EA7
:101520009574F50EE50D9573F50DE50C9572F50CBA
:10153000E50B9571F50B800312113DE47F607EEAA7
:10154000FDFC121182400BE4750E60750DEAF50C7E
:10155000F50BAE0DAF0E2290017DE0FEA3E0FFC3C0
:101560009404EE9400502F900106E0FCA3E0FDEF00
:1015700025E0FFEE33FE74752FF58274013EF5838E
:10158000ECF0A3EDF090017EE004F0700690017D98
:10159000E004F0021DFC750D011210C9E50D25E0F7
:1015A0002473F582E43401F583EEF0A3EFF0050D2A
:1015B000E50DB404E4120FE1FF9001061210E8E516
:1015C000F09CFE12084EC3EF9428EE648094805085
:1015D0003C900132E0702890010E120FE4FFC3909E
:1015E0000107E09FFF900106E095F0FE12084EC350
:1015F000EF9414EE64809480500590010E80039067
:101600000108120FE4FF90017BE5F0800B900106CA
:10161000E0FFA3E090017BCFF0A3EFF0E4F50CF541
:101620000BF50AF509F50DD390017EE0950D9001BB
:101630007DE09400401E1210C9E4FCFDE50C2FF57E
:101640000CE50B3EF50BED350AF50AEC3509F5090D
:10165000050D80D3AF0CAE0BAD0AAC09EEC0E0EFC8
:10166000C0E090017D121080D0E0FFD0E0FE120AB1
:10167000908F0C8E0B8D0A8C0922C0E0C083C08233
:10168000C0D0ECC0E0EDC0E0EEC0E0EFC0E0D2AF13
:10169000E5DB30E419D20CC208E5DB30E102802E34
:1016A0009002D7E5DFF09002DAE4F0021F58E5DBA4
:1016B00030E50FD206300805C208021F58C20C02DE
:1016C0001F58C208E5DB30E13AE5DB30E01090025C
:1016D000DBE0FF04F0122C2BE0F5DF021F58900234
:1016E000DBE0FFB40813208A10D28A9002D8E0FC15
:1016F000A3E02407122C31E4F0EF641A707AD207C9
:10170000021F589002DAE0700EA3E5DFF09002DAD3
:101710007401F0D20880619002DBE0902A0893FF08
:10172000B4FF089002D7E5DFF08047EF640F70291F
:101730009002DBE0FFA3E0FCA3E0FD122C30E054BC
:101740000FF09002DBE0FF04F0ED122C30E0FFE53B
:10175000DF54F0FEEF4EF0801F9002DBE0FF122C12
:101760002BE5DFF0EFB4240A9002147401F0A374A7
:10177000F4F09002DBE004F075DBFFD0E0FFD0E096
:10178000FED0E0FDD0E0FCD0D0D082D083D0E032DB
:101790009002CAEFF09002CFE4F0A374FFF0E4A34C
:1017A000F0A3F0A304F0A374FFF0902EC07402F035
:1017B000902EC37408F0E49002CBF0A3F09002CB1B
:1017C000E0FEA3E0FFC39409EE9400400302205F13
:1017D000EF9407EE940040067E007F01801990028E
:1017E000CBA3E004FFE47E01C8EFC8088006CEA2C8
:1017F000E713CE13D8F8FF9002CDEEF0A3EFF090F0
:101800002EC07419F0902EC0E030E2F99002CAE0C8
:10181000FF75F002A424001229E4E0FCA3E0FD908F
:101820002EC07402F0D3ED94FFEC940F4017900299
:10183000CDE0FCA3E0FD75F002EF1229E1EC8DF0A4
:101840001209BC80299002CAE075F0021229E1C099
:1018500083C082E0FEA3E0FF9002CDE0FCA3E0FDA8
:10186000C3EF9DFFEE9CD082D083F0A3EFF09002F7
:10187000CCE004F070069002CBE004F0021F9D7FE4
:1018800000227F997A0179061210509001087401A4
:10189000F0A37400F0744412102E7400F074461219
:1018A000102E7400F0A3744812102F7400F0A3746B
:1018B0003212102F7400F0A3742E12102F7400F047
:1018C000A3742CF09001237401F0A37400F0A374AE
:1018D00026F09001987401F0A37400F0A3748412B0
:1018E000102F7400F0A37486F09001267401F0A309
:1018F0007400F0A3741C12102F7400F0A37422F073
:1019000090011A7401F0A37400F0A3743612102F22
:101910007400F0A3742A12102F7400F0A37438F02E
:10192000757900757AC890011A120FFCF9E579856E
:101930007AF0120A3590011D120FFCF9E475F0647B
:10194000120A35900120120FFCF9E475F096020A94
:1019500035122B22902E42E0FEA3E0249CFFEE34B1
:10196000FE9002C8F0A3EFF012102153997F122AC3
:101970003E120866902EC07402F0902EC314F0122E
:1019800010C2902EC0E030E2F9902EC0E4F0902E0C
:10199000027D121210918E268F277D14120B99EF63
:1019A00024E0F574EE34B1F573ED34FFF572EC34E8
:1019B000FFF5714389021210274380024399805337
:1019C000997F120870902E5EE4F0A374FFF07F0FF1
:1019D000121F70902E5EE0FEA3E0D394F0EE94010F
:1019E0004007902E5EE4F0A3F0902EC4E4F04399FB
:1019F00080A3F0900105E0900021F012108C90017E
:101A000026120FFCF9EE8FF0020A359002CCEEF0B0
:101A1000A3EFF0E5644563700C9002CCE0F563A39E
:101A2000E0F56480169002CDE02564FF9002CCE0E2
:101A300035631211E2F563EF13F5640565E565D3CF
:101A4000940A400D856361856462E4F563F564F58D
:101A500065D3E5629400E5619400405C9002CDE0BE
:101A60009562FF9002CCE09561FE12084EC3EF94A0
:101A70000AEE648094805028AE61AF627C007D03E2
:101A800012112D9002CCE0FEA3E0FFE4FCFDEB2F51
:101A9000FFEA3E12106C7802120B499002CC8013C0
:101AA0009002CDE02562FF9002CCE03561C313FEC9
:101AB000EF13FFEEF0A3EFF09002CCE0FEA3E0FF07
:101AC000229002C6EEF0A3EF1211159002C6E0704C
:101AD00002A3E060031221311226BFE490017DF0E1
:101AE000A3F07F14122A70121074A312118E9001A9
:101AF00006E0F9A3E0FFA3120FFC12103690010BD1
:101B0000120FFC1210B1900111120FFC1211C890AB
:101B10000114120FFC1210B1900117120FFC1211D8
:101B2000C81211D1E4900132F0900134120B680018
:101B3000000000E490013812110EF0900106120F1F
:101B4000F4121036E4900133F09002221211D89072
:101B5000021EF0A3F0FE7F14FD7B017A017984124E
:101B60000BC6900123120FE490018A1211259001F7
:101B70009212117B22022ACBE493A3F8E493A340B0
:101B800003F68001F208DFF48029E493A3F85407F8
:101B9000240CC8C333C4540F4420C8834004F456F3
:101BA000800146F6DFE4800B01020408102040802B
:101BB000902545E47E019360BCA3FF543F30E509C6
:101BC000541FFEE493A360010ECF54C025E060A82B
:101BD00040B8E493A3FAE493A3F8E493A3C8C582BE
:101BE000C8CAC583CAF0A3C8C582C8CAC583CADF2C
:101BF000E9DEE780BE30000875791B757A588006EB
:101C0000757900757AC890010B120FE4FFAEF0C32E
:101C1000957AEE95795015900132E0602090012080
:101C2000120FE4FDC3EF9DEE95F0401190021AE013
:101C30007002A3E0702790013204F0802090001B16
:101C4000E0B420051211C0800690021A12117BE444
:101C5000900132F0900218F0A3F01211D1900132ED
:101C6000E06011900028E090003AB410047410F085
:101C7000227420F02290022FE014601B1460432491
:101C800002705D900239E0B4010A90022F1224C163
:101C9000D205D200C203227F021228D6EF60077F4E
:101CA0000212085AC205900239E0703490022F7473
:101CB00002F0D203C205C2007F0312085A7F03025A
:101CC00027717F031228D6EF60167F0312085A90FF
:101CD0000239E090022F7003F080031224C1C20386
:101CE000227401F07F0212085A7F0212277122CD5E
:101CF000EFCD43AD105399EF439A10539BEF902EC5
:101D0000C07402F0147E00C8EDC8088005C333CE4D
:101D100033CED8F9FF902EC4EEF0A3EFF0902EC88A
:101D2000EEF0A3EFF07410122B7E902EC0E030E2A4
:101D3000F9902EC0E4F07402F07420122B7E902EE5
:101D4000C0E030E2F9902E00E0FEA3E0FF902EC448
:101D5000E4F0A3F0902EC0F0439910539AEF539BF8
:101D6000EF5390EF22C10C41023300410234004195
:101D700002300041023800C102C101C104410239F0
:101D80000041022F00C103C100C1054102DA004138
:101D900002DB004202D50000C106C108C1074102B2
:101DA000D7104101030041010510C10BC10A4101D7
:101DB0009F00022600000471000000004101041091
:101DC00041023A00009002C47408F0A3E4F0A37446
:101DD0003FF0A374DFF0E4FDFCF9758A10538AEF3D
:101DE000009002C4E0FEA3E02DF582EE3CF583E412
:101DF00093FF69F90DBD00010CBC37E5BDDFE29032
:101E000002C6122C38E493699002D87009122C385B
:101E1000A3740BF08006122C38A3E4F0758A50539B
:101E20008AEF0022200A06200303300509E4FFFEA2
:101E30001222A1C20A22900220E07002A3E06005F3
:101E400012114E703A2000031229581226BF7F014A
:101E5000122A70121D379002C4EEF0A3EFF07B013E
:101E60007A0279C412280A9002C41210F7120FFCE9
:101E70001210361213E91223D512120F12178A12FA
:101E8000299422900211E024FE6013146023146050
:101E900027240370499002117402F0122C477F012D
:101EA0007E001222A19002117403F0E4900230F03F
:101EB000229002117404F0221224551227C2122417
:101EC00055900171E07004A3E06401700C90017101
:101ED000F0A3F09002117402F0E4900225F0224386
:101EE00089025395FD5396FD438002122BB87F0C57
:101EF0001224CFCAEECACBEFCB7F0C1224CFEF2B2C
:101F0000FFEE3A9002C9F0A3EFF0122B8AF9120902
:101F1000D245F07006122B6FEE80181209D2FBAA80
:101F2000F0122B6FEF2BFFEE3AC313F9EF13FF12F2
:101F30002B8AC98FF0120A35221229EDF5828E8381
:101F4000A3E0B4AA031225A51229EDFF1229D8E0B7
:101F5000B41008EF1229D8E4F0D20A1229EDFF24B8
:101F60001B1229DAE0700DEF241C1229DAE0B410FC
:101F7000031228511229ED24131229DAE0FFB410BC
:101F8000069002397401F0EFB42005E4900239F0B4
:101F9000229002C4EFF0E024BB122B98E060037F94
:101FA00001229002C4E0FF24BB122B987401F0EFD1
:101FB000122BA0E493FE740193FFE4FCFD902F60CC
:101FC000E0F8A3E0F9A3E0FAA3E02FFFEA3EFEED7C
:101FD00039EC389002C4E0122BACEEF0A3EFF07FA6
:101FE000002212114E702990019FE07003121074AC
:101FF00090019F7401F0900029E0B420081226049B
:10200000120C478003122A9E9002247401F080175C
:10201000E490019FF0900029E0B420031226049080
:102020000224E06002E4F0022BDB9002C6EBF0A396
:10203000EAF0A3E9F0900214E07002A3E07031909E
:102040000133E0602BE4900133F01226BF121074CC
:102050007508017F01122A70121D379002C6120FF7
:10206000FC1210B80508E508C3941440E61211C02C
:102070002212082EE4F5F275F30875EEFF75EF3FB6
:1020800075EA81F5F675EB0700E5EC30E7FBE4F562
:10209000EC9002D8E0FEA3E0FF241BF582E43EF5BD
:1020A00083E5F3F0EF241CF582E43EF583E5F2F0DE
:1020B00075EB3022758B11902F647440F0E4FEE4D0
:1020C000FFEF75F003A4244DF582E43402F583E5B7
:1020D000822EF582E43583F583E4F00FEFB40AE154
:1020E0000EEEB403DA7F099002BBE4F0A3DFFC90AC
:1020F0002F647480F022CBEFCB122B95E0603690EA
:102100002F60A3A3E0FEA3E0FFEB122BACE0FCA347
:10211000E0FDD39FEC9E501DC3EF9DFFEE9CFEEBB8
:10212000122BA0C37401939FE4939E4008122B9539
:10213000E4F07F01227F0022758A50538AEF9000DD
:10214000027411F09000017422F09000037433F0D7
:10215000E4F5AB75AC1DF5ADF5AF7589FF75913F35
:102160007599FFF59675931CF59BF595F592F59A83
:102170005388FCD28AD20D22300738C207902E42F3
:10218000E0FFA3E09002C6CFF0A3EFF0122B2212E3
:10219000108C900126120FFC1210B8902EC0740201
:1021A000F09002C6E0FFA3E0902E42CFF0A3EFF044
:1021B0001210742290003AE0FC900104E06C602E52
:1021C00090003AE0FE900104F090000BE09002389D
:1021D000F0540FF0EEB42005E04420800AECB41077
:1021E0000B900238E04410F090000BF0C28A22F508
:1021F00082E43CF583EFF022241AF582E43EF58375
:1022000022A42440F582E5F0342EF583229002D8F2
:10221000E0FEA3E022A3F0A37401F0A322746A2FCE
:10222000F582E43400F5832200000000FFFFFFFF89
:102230000000FFFFFFFFFFFFFFFFFF00FF000000A8
:10224000FFFF000000FFFFFFFFFFFFFF0000000097
:10225000FFFFFFFFFFFFFFFFFFFF00000000121165
:1022600064FF74542FF582E43400F583E0FE75F0CA
:1022700002EFA42400F582E5F0342EF583E49324E4
:10228000C0F582E4342EF583EEF00FEFB416D322BE
:102290009002C9EFF0122A3EE4F5099002C9E0FF6E
:1022A000E509C39F50071215BD050980EE902EC0A9
:1022B000E4F0121BFA900106EEF0A3EFF022E4F531
:1022C000B2F5BA758D20438D20538D7F53AAF7F553
:1022D0008BE5DB20E211200C0EE4F58A7587030004
:1022E0000000758A50D20A758B1122122C1553A842
:1022F0007F12291812081E122AF743A880122C41B7
:102300009000FFE060069002117401F0122BF912A8
:10231000271912266380F59002D8E0FFA3E090020F
:10232000DCCFF0A3EFF0E4F5DA75DA4043DA20759C
:10233000D74075DA5875D90143A90875B80875F8FA
:10234000082212102153997F122A3E902E42E4F067
:10235000A374FFF01208667F01121F7043890212F6
:1023600010274380024399802201F40028002801AD
:10237000F4009603E801F403E81770006403E80032
:102380003202580258012C01F403E8271000C890CB
:1023900002C9E0FEA3E0FF7C007D14020974902EC8
:1023A000C2F0902EC0E04419F022900123E0FBA37C
:1023B000E0FAA3E02274BB2BF582E43402F5832219
:1023C00025E0245DF582E4342BF5832225E0243BCF
:1023D000F582E43402F58322902EC07402F0902E30
:1023E000C77474F0902ECD74C0F0A374FFF0A3F006
:1023F000902EC37401F0902ECAF022E5B230E005B1
:10240000E5AA20E013E4900226F075B28E75B6F9C5
:10241000F5B743B20143AA0122E4FF300616900249
:10242000D8E0FCA3E0F5828C83E0FE54F0FFEE548C
:102430000FF0C2062290407FE493FF64326003EF06
:102440007002002253A87F000080FCA3E0FCA3E000
:102450002FF582E43CF58322E0FEA3E0F5828E8333
:1024600022122C510228941211D122D2AF32D2AFB3
:1024700032022BDB00000000000000000000000022
:10248000000000000000000000000000000000004C
:10249000000000000000000000000000000000003C
:1024A000000000000000000000000000000000002C
:1024B000000000000000000000000000000000001C
:1024C000000000000000000000000000000000000C
:1024D00000000000000000000000000000000000FC
:1024E00000000000000000000000000000000000EC
:1024F00000000000000000000000000000000000DC
:1025000000000000000000000000000000000000CB
:1025100000000000000000000000000000000000BB
:1025200000000000000000000000000000000000AB
:10253000000000000000000000000000000000009B
:10254000000000000000000000000000000000008B
:10255000000000000000000000000000000000007B
:10256000000000000000000000000000000000006B
:10257000000000000000000000000000000000005B
:10258000000000000000000000000000000000004B
:10259000000000000000000000000000000000003B
:1025A000000000000000000000000000000000002B
:1025B000000000000000000000000000000000001B
:1025C000000000000000000000000000000000000B
:1025D00000000000000000000000000000000000FB
:1025E00000000000000000000000000000000000EB
:1025F00000000000000000000000000000000000DB
:102600000B05AB62000000000000000000000000AD
:1026100000000000000000000000000000000000BA
:10262000021203030A140DA00EB60FFF0C020BFFDB
:1026300023F724062504070127082A0828022B026D
:1026400029032C032D082E082F0426080211030647
:102650000A100D400E800FFF0C020BFF23F4240420
:102660002504070127102A1028042B0429032C0312
:102670002D202E202F10262000000000000000003A
:10268000000000000000000000000000000000004A
:10269000000000000000000000000000000000003A
:1026A000000000000000000000000000000000002A
:1026B000000000000000000000000000000000001A
:1037F0000000000000000000000000000000009732
:1038000000000000000000000000000000000000B8
:1038100000000000000000000000000000000000A8
:00000001FF
